 HDA

 Timestamp is 697a6ddd (Wed Jan 28 12:13:17 2026)

 Preferred load address is 00010000

 Start         Length     Name                   Class
 0001:00000000 00003ebcH .text                   CODE
 0002:00000000 000000b8H .idata$5                DATA
 0002:000000b8 00000630H .rdata                  DATA
 0003:00000000 00000d18H .data                   DATA
 0003:00000d18 00000016H .bss                    DATA
 0004:00000000 0000c200H PAGE                    CODE
 0005:00000000 000000a9H INIT                    CODE
 0005:000000ac 0000003cH .idata$2                CODE
 0005:000000e8 00000014H .idata$3                CODE
 0005:000000fc 000000b8H .idata$4                CODE
 0005:000001b4 000003b4H .idata$6                CODE
 0006:00000000 00000058H .rsrc$01                DATA
 0006:00000060 000003d8H .rsrc$02                DATA

  Address         Publics by Value              Rva+Base     Lib:Object

 0001:00000000       ??3@YAXPAX@Z               000102e0 f i common.obj
 0001:00000010       ??2@YGPAXIW4_POOL_TYPE@@K@Z 000102f0 f i common.obj
 0001:00000050       ??0CAdapterCommon@@QAE@PAUIUnknown@@@Z 00010330 f i common.obj
 0001:000000a0       ?QueryInterface@CAdapterCommon@@UAGJABU_GUID@@PAPAX@Z 00010380 f i common.obj
 0001:000000d0       ?GetOuterUnknown@CUnknown@@QAEPAUIUnknown@@XZ 000103b0 f i common.obj
 0001:000000f0       ?AddRef@CAdapterCommon@@UAGKXZ 000103d0 f i common.obj
 0001:00000120       ?Release@CAdapterCommon@@UAGKXZ 00010400 f i common.obj
 0001:00000150       ??_GCAdapterCommon@@UAEPAXI@Z 00010430 f i common.obj
 0001:00000150       ??_ECAdapterCommon@@UAEPAXI@Z 00010430 f i common.obj
 0001:00000190       ??0IUnknown@@QAE@XZ        00010470 f i common.obj
 0001:000001a0       _IsEqualGUIDAligned@8      00010480 f i common.obj
 0001:00000220       ?hda_check_headphone_connection_change@CAdapterCommon@@QAGXXZ 00010500 f   common.obj
 0001:00000312       ?hda_is_supported_sample_rate@CAdapterCommon@@UAGEK@Z 000105f2 f   common.obj
 0001:00000496       ?hda_send_verb@CAdapterCommon@@QAGKKKKK@Z 00010776 f   common.obj
 0001:00000792       ?ReadController@CAdapterCommon@@UAGEXZ 00010a72 f   common.obj
 0001:00000836       ?WriteController@CAdapterCommon@@UAGEE@Z 00010b16 f   common.obj
 0001:00000942       ?MixerRegWrite@CAdapterCommon@@UAGXEE@Z 00010c22 f   common.obj
 0001:00000b2a       ?MixerRegRead@CAdapterCommon@@UAGEE@Z 00010e0a f   common.obj
 0001:00000c0e       ?MixerReset@CAdapterCommon@@UAGXXZ 00010eee f   common.obj
 0001:00000cae       ?AcknowledgeIRQ@CAdapterCommon@@AAE?AW4_HDA_INTERRUPT_TYPE@@XZ 00010f8e f   common.obj
 0001:00000f52       ?ResetController@CAdapterCommon@@UAGJXZ 00011232 f   common.obj
 0001:00000ff6       ?RestoreMixerSettingsFromRegistry@CAdapterCommon@@UAGJXZ 000112d6 f   common.obj
 0001:000012a2       ?SaveMixerSettingsToRegistry@CAdapterCommon@@UAGJXZ 00011582 f   common.obj
 0001:0000168a       ?ProgramSampleRate@CAdapterCommon@@UAGJK@Z 0001196a f   common.obj
 0001:00001b06       ?PowerChangeState@CAdapterCommon@@UAGXT_POWER_STATE@@@Z 00011de6 f   common.obj
 0001:00001cf6       ?QueryPowerChangeState@CAdapterCommon@@UAGJT_POWER_STATE@@@Z 00011fd6 f   common.obj
 0001:00001d7a       ?QueryDeviceCapabilities@CAdapterCommon@@UAGJPAU_DEVICE_CAPABILITIES@@@Z 0001205a f   common.obj
 0001:00001e2a       ?InterruptServiceRoutine@@YGJPAUIInterruptSync@@PAX@Z 0001210a f   common.obj
 0001:00001fb6       ?hda_stop_stream@CAdapterCommon@@UAGJXZ 00012296 f   common.obj
 0001:00002230       ?hda_start_sound@CAdapterCommon@@UAGXXZ 00012510 f   common.obj
 0001:0000229a       ?hda_stop_sound@CAdapterCommon@@UAGXXZ 0001257a f   common.obj
 0001:00002396       ?hda_get_actual_stream_position@CAdapterCommon@@UAGKXZ 00012676 f   common.obj
 0001:00002490       ?hda_set_volume@CAdapterCommon@@QAGXKE@Z 00012770 f   common.obj
 0001:00002500       ?hda_set_node_gain@CAdapterCommon@@QAGXKKKKKE@Z 000127e0 f   common.obj
 0001:000025a0       ?readUCHAR@CAdapterCommon@@QAGEG@Z 00012880 f   common.obj
 0001:000025c0       ?writeUCHAR@CAdapterCommon@@QAGXGE@Z 000128a0 f   common.obj
 0001:000025f0       ?readUSHORT@CAdapterCommon@@QAGGG@Z 000128d0 f   common.obj
 0001:00002610       ?writeUSHORT@CAdapterCommon@@QAGXGG@Z 000128f0 f   common.obj
 0001:00002640       ?readULONG@CAdapterCommon@@QAGKG@Z 00012920 f   common.obj
 0001:00002660       ?writeULONG@CAdapterCommon@@QAGXGK@Z 00012940 f   common.obj
 0001:0000283a       ?hda_showtime@CAdapterCommon@@UAGJPAUIDmaChannel@@@Z 00012b1a f   common.obj
 0001:00002cc0       ?hda_return_sound_data_format@CAdapterCommon@@QAGGKKK@Z 00012fa0 f   common.obj
 0001:00002e30       ?ReadWriteConfigSpace@CAdapterCommon@@AAGJPAU_DEVICE_OBJECT@@KPAXKK@Z 00013110 f   common.obj
 0001:00002f5b       ?WriteConfigSpaceByte@CAdapterCommon@@AAGJEEE@Z 0001323b f   common.obj
 0001:0000305b       ?WriteConfigSpaceWord@CAdapterCommon@@AAGJEGG@Z 0001333b f   common.obj
 0001:00003120       ?QueryInterface@CAdapterCommon@@W3AGJABU_GUID@@PAPAX@Z 00013400 f i common.obj
 0001:00003130       ?AddRef@CAdapterCommon@@W3AGKXZ 00013410 f i common.obj
 0001:00003140       ?Release@CAdapterCommon@@W3AGKXZ 00013420 f i common.obj
 0001:00003150       ??0CMiniportTopologyHDA@@QAE@PAUIUnknown@@@Z 00013430 f i mintopo.obj
 0001:00003190       ?QueryInterface@CMiniportWaveCyclicHDA@@UAGJABU_GUID@@PAPAX@Z 00013470 f i mintopo.obj
 0001:00003190       ?QueryInterface@CMiniportWaveCyclicStreamHDA@@UAGJABU_GUID@@PAPAX@Z 00013470 f i mintopo.obj
 0001:00003190       ?QueryInterface@CMiniportTopologyHDA@@UAGJABU_GUID@@PAPAX@Z 00013470 f i mintopo.obj
 0001:000031c0       ?DataRangeIntersection@CMiniportTopologyHDA@@UAGJKPATKSDATAFORMAT@@0KPAXPAK@Z 000134a0 f i mintopo.obj
 0001:000031d0       ??_GCMiniportTopologyHDA@@UAEPAXI@Z 000134b0 f i mintopo.obj
 0001:000031d0       ??_ECMiniportTopologyHDA@@UAEPAXI@Z 000134b0 f i mintopo.obj
 0001:00003890       ?ReadBitsFromMixer@CMiniportTopologyHDA@@AAEEEEE@Z 00013b70 f   mintopo.obj
 0001:000038e0       ?ThisManyOnes@@YGEE@Z      00013bc0 f i mintopo.obj
 0001:00003900       ?WriteBitsToMixer@CMiniportTopologyHDA@@AAEXEEEE@Z 00013be0 f   mintopo.obj
 0001:000039a0       ??0CMiniportWaveCyclicHDA@@QAE@PAUIUnknown@@@Z 00013c80 f i minwave.obj
 0001:000039e0       ?AddRef@CMiniportTopologyHDA@@UAGKXZ 00013cc0 f i minwave.obj
 0001:000039e0       ?AddRef@CMiniportWaveCyclicStreamHDA@@UAGKXZ 00013cc0 f i minwave.obj
 0001:000039e0       ?AddRef@CMiniportWaveCyclicHDA@@UAGKXZ 00013cc0 f i minwave.obj
 0001:00003a10       ??_ECMiniportWaveCyclicHDA@@UAEPAXI@Z 00013cf0 f i minwave.obj
 0001:00003a10       ??_GCMiniportWaveCyclicHDA@@UAEPAXI@Z 00013cf0 f i minwave.obj
 0001:00003a50       ??0IMiniportTopology@@QAE@XZ 00013d30 f i minwave.obj
 0001:00003a50       ??0IMiniportWaveCyclic@@QAE@XZ 00013d30 f i minwave.obj
 0001:00003a70       ??2@YGPAXIW4_POOL_TYPE@@@Z 00013d50 f i minwave.obj
 0001:00003ac0       ??0CMiniportWaveCyclicStreamHDA@@QAE@PAUIUnknown@@@Z 00013da0 f i minwave.obj
 0001:00003b00       ?Release@CMiniportWaveCyclicStreamHDA@@UAGKXZ 00013de0 f i minwave.obj
 0001:00003b00       ?Release@CMiniportTopologyHDA@@UAGKXZ 00013de0 f i minwave.obj
 0001:00003b00       ?Release@CMiniportWaveCyclicHDA@@UAGKXZ 00013de0 f i minwave.obj
 0001:00003b30       ??_GCMiniportWaveCyclicStreamHDA@@UAEPAXI@Z 00013e10 f i minwave.obj
 0001:00003b30       ??_ECMiniportWaveCyclicStreamHDA@@UAEPAXI@Z 00013e10 f i minwave.obj
 0001:00003b70       ??0IAdapterPowerManagement@@QAE@XZ 00013e50 f i minwave.obj
 0001:00003b70       ??0IMiniportWaveCyclicStream@@QAE@XZ 00013e50 f i minwave.obj
 0001:00003b70       ??0IAdapterCommon@@QAE@XZ  00013e50 f i minwave.obj
 0001:00003b70       ??0IMiniport@@QAE@XZ       00013e50 f i minwave.obj
 0001:00003ba9       ?GetPosition@CMiniportWaveCyclicStreamHDA@@UAGJPAK@Z 00013e89 f   minwave.obj
 0001:00003c9e       ?NormalizePhysicalPosition@CMiniportWaveCyclicStreamHDA@@UAGJPA_J@Z 00013f7e f   minwave.obj
 0001:00003d40       ?Silence@CMiniportWaveCyclicStreamHDA@@UAGXPAXK@Z 00014020 f   minwave.obj
 0001:00003d7e       _DbgPrint                  0001405e f   ntoskrnl:ntoskrnl.exe
 0001:00003d84       _DbgBreakPoint@0           00014064 f   ntoskrnl:ntoskrnl.exe
 0001:00003d8a       __alldiv                   0001406a f   ntoskrnl:ntoskrnl.exe
 0001:00003d90       __allmul                   00014070 f   ntoskrnl:ntoskrnl.exe
 0001:00003d96       _PcInitializeAdapterDriver@12 00014076 f   portcls:portcls.sys
 0001:00003d9c       _PcAddAdapterDevice@20     0001407c f   portcls:portcls.sys
 0001:00003da2       _PcRegisterSubdevice@12    00014082 f   portcls:portcls.sys
 0001:00003da8       _PcNewMiniport@8           00014088 f   portcls:portcls.sys
 0001:00003dae       _PcNewPort@8               0001408e f   portcls:portcls.sys
 0001:00003db4       _PcRegisterPhysicalConnection@20 00014094 f   portcls:portcls.sys
 0001:00003dba       _PcRegisterAdapterPowerManagement@8 0001409a f   portcls:portcls.sys
 0001:00003dc0       _PcNewResourceSublist@20   000140a0 f   portcls:portcls.sys
 0001:00003dc6       _PcNewInterruptSync@20     000140a6 f   portcls:portcls.sys
 0001:00003dcc       _PcNewRegistryKey@36       000140ac f   portcls:portcls.sys
 0001:00003dd2       _PcNewServiceGroup@8       000140b2 f   portcls:portcls.sys
 0001:00003dd8       ??0CUnknown@@QAE@PAUIUnknown@@@Z 000140b8 f   stdunk:stdunk.obj
 0001:00003df7       ??_GCUnknown@@UAEPAXI@Z    000140d7 f i stdunk:stdunk.obj
 0001:00003df7       ??_ECUnknown@@UAEPAXI@Z    000140d7 f i stdunk:stdunk.obj
 0001:00003e13       ??1CUnknown@@UAE@XZ        000140f3 f   stdunk:stdunk.obj
 0001:00003e1a       ?NonDelegatingAddRef@CUnknown@@UAGKXZ 000140fa f   stdunk:stdunk.obj
 0001:00003e30       ?NonDelegatingRelease@CUnknown@@UAGKXZ 00014110 f   stdunk:stdunk.obj
 0001:00003e5f       ?NonDelegatingQueryInterface@CUnknown@@UAGJABU_GUID@@PAPAX@Z 0001413f f   stdunk:stdunk.obj
 0002:00000000       __imp_@KfAcquireSpinLock@4 000141a0     hal:HAL.dll
 0002:00000004       __imp_@KfReleaseSpinLock@8 000141a4     hal:HAL.dll
 0002:00000008       __imp__KeStallExecutionProcessor@4 000141a8     hal:HAL.dll
 0002:0000000c       __imp__KeGetCurrentIrql@0  000141ac     hal:HAL.dll
 0002:00000010       \177HAL_NULL_THUNK_DATA    000141b0     hal:HAL.dll
 0002:00000014       __imp__MmMapIoSpace@16     000141b4     ntoskrnl:ntoskrnl.exe
 0002:00000018       __imp__KeInitializeSpinLock@4 000141b8     ntoskrnl:ntoskrnl.exe
 0002:0000001c       __imp__MmUnmapIoSpace@8    000141bc     ntoskrnl:ntoskrnl.exe
 0002:00000020       __imp__IoGetDmaAdapter@12  000141c0     ntoskrnl:ntoskrnl.exe
 0002:00000024       __imp__RtlInitUnicodeString@8 000141c4     ntoskrnl:ntoskrnl.exe
 0002:00000028       __imp__READ_REGISTER_ULONG@4 000141c8     ntoskrnl:ntoskrnl.exe
 0002:0000002c       __imp__WRITE_REGISTER_ULONG@8 000141cc     ntoskrnl:ntoskrnl.exe
 0002:00000030       __imp__READ_REGISTER_UCHAR@4 000141d0     ntoskrnl:ntoskrnl.exe
 0002:00000034       __imp__WRITE_REGISTER_UCHAR@8 000141d4     ntoskrnl:ntoskrnl.exe
 0002:00000038       __imp__READ_REGISTER_USHORT@4 000141d8     ntoskrnl:ntoskrnl.exe
 0002:0000003c       __imp__ExFreePool@4        000141dc     ntoskrnl:ntoskrnl.exe
 0002:00000040       __imp__ExAllocatePoolWithTag@12 000141e0     ntoskrnl:ntoskrnl.exe
 0002:00000044       __imp__KeWaitForSingleObject@20 000141e4     ntoskrnl:ntoskrnl.exe
 0002:00000048       __imp_@IofCallDriver@8     000141e8     ntoskrnl:ntoskrnl.exe
 0002:0000004c       __imp__IoBuildSynchronousFsdRequest@28 000141ec     ntoskrnl:ntoskrnl.exe
 0002:00000050       __imp__IoGetAttachedDeviceReference@4 000141f0     ntoskrnl:ntoskrnl.exe
 0002:00000054       __imp__KeInitializeEvent@12 000141f4     ntoskrnl:ntoskrnl.exe
 0002:00000058       __imp__KeInitializeMutex@8 000141f8     ntoskrnl:ntoskrnl.exe
 0002:0000005c       __imp__RtlAssert@16        000141fc     ntoskrnl:ntoskrnl.exe
 0002:00000060       __imp___alldiv             00014200     ntoskrnl:ntoskrnl.exe
 0002:00000064       __imp___allmul             00014204     ntoskrnl:ntoskrnl.exe
 0002:00000068       __imp__DbgBreakPoint@0     00014208     ntoskrnl:ntoskrnl.exe
 0002:0000006c       __imp__DbgPrint            0001420c     ntoskrnl:ntoskrnl.exe
 0002:00000070       __imp_@ObfDereferenceObject@4 00014210     ntoskrnl:ntoskrnl.exe
 0002:00000074       __imp__WRITE_REGISTER_USHORT@8 00014214     ntoskrnl:ntoskrnl.exe
 0002:00000078       __imp__KeReleaseMutex@8    00014218     ntoskrnl:ntoskrnl.exe
 0002:0000007c       __imp_@InterlockedDecrement@4 0001421c     ntoskrnl:ntoskrnl.exe
 0002:00000080       __imp_@InterlockedIncrement@4 00014220     ntoskrnl:ntoskrnl.exe
 0002:00000084       \177ntoskrnl_NULL_THUNK_DATA 00014224     ntoskrnl:ntoskrnl.exe
 0002:00000088       __imp__PcInitializeAdapterDriver@12 00014228     portcls:portcls.sys
 0002:0000008c       __imp__PcNewMiniport@8     0001422c     portcls:portcls.sys
 0002:00000090       __imp__PcNewPort@8         00014230     portcls:portcls.sys
 0002:00000094       __imp__PcRegisterPhysicalConnection@20 00014234     portcls:portcls.sys
 0002:00000098       __imp__PcAddAdapterDevice@20 00014238     portcls:portcls.sys
 0002:0000009c       __imp__PcRegisterSubdevice@12 0001423c     portcls:portcls.sys
 0002:000000a0       __imp__PcNewInterruptSync@20 00014240     portcls:portcls.sys
 0002:000000a4       __imp__PcNewRegistryKey@36 00014244     portcls:portcls.sys
 0002:000000a8       __imp__PcNewServiceGroup@8 00014248     portcls:portcls.sys
 0002:000000ac       __imp__PcRegisterAdapterPowerManagement@8 0001424c     portcls:portcls.sys
 0002:000000b0       __imp__PcNewResourceSublist@20 00014250     portcls:portcls.sys
 0002:000000b4       \177portcls_NULL_THUNK_DATA 00014254     portcls:portcls.sys
 0002:00000130       _IID_IAdapterCommon        000142d0     adapter.obj
 0002:00000140       _CLSID_MiniportDriverFmSynth 000142e0     adapter.obj
 0002:00000150       _CLSID_PortWaveCyclic      000142f0     adapter.obj
 0002:00000160       _CLSID_PortTopology        00014300     adapter.obj
 0002:00000170       _CLSID_PortMidi            00014310     adapter.obj
 0002:00000180       _IID_IAdapterPowerManagment 00014320     adapter.obj
 0002:00000190       _IID_IMiniportWaveCyclicStream 00014330     adapter.obj
 0002:000001a0       _IID_IMiniportWaveCyclic   00014340     adapter.obj
 0002:000001b0       _IID_IPortWaveCyclic       00014350     adapter.obj
 0002:000001c0       _IID_IMiniportTopology     00014360     adapter.obj
 0002:000001d0       _IID_IMiniport             00014370     adapter.obj
 0002:000001e0       _IID_IUnknown              00014380     adapter.obj
 0002:000001f0       ??_C@_1BE@FFBG@?$AAU?$AAs?$AAe?$AAD?$AAm?$AAa?$AAP?$AAo?$AAs?$AA?$AA@ 00014390     common.obj
 0002:00000204       ??_C@_1CA@DADJ@?$AAU?$AAs?$AAe?$AAD?$AAi?$AAs?$AAa?$AAb?$AAl?$AAe?$AAd?$AAP?$AAi?$AAn?$AAs?$AA?$AA@ 000143a4     common.obj
 0002:00000224       ??_C@_1BC@MBIB@?$AAU?$AAs?$AAe?$AAS?$AAP?$AAD?$AAI?$AAF?$AA?$AA@ 000143c4     common.obj
 0002:00000238       ??_C@_1BE@ONOC@?$AAU?$AAs?$AAe?$AAA?$AAl?$AAt?$AAO?$AAu?$AAt?$AA?$AA@ 000143d8     common.obj
 0002:0000024c       ??_C@_1BO@LMMA@?$AAS?$AAk?$AAi?$AAp?$AAC?$AAo?$AAd?$AAe?$AAc?$AAR?$AAe?$AAs?$AAe?$AAt?$AA?$AA@ 000143ec     common.obj
 0002:0000026c       ??_C@_1CI@JKGI@?$AAS?$AAk?$AAi?$AAp?$AAC?$AAo?$AAn?$AAt?$AAr?$AAo?$AAl?$AAl?$AAe?$AAr?$AAR?$AAe?$AAs?$AAe?$AAt?$AA?$AA@ 0001440c     common.obj
 0002:00000294       ??_C@_1BE@ENEK@?$AAR?$AAi?$AAg?$AAh?$AAt?$AAB?$AAa?$AAs?$AAs?$AA?$AA@ 00014434     common.obj
 0002:000002a8       ??_C@_1BC@JMJO@?$AAL?$AAe?$AAf?$AAt?$AAB?$AAa?$AAs?$AAs?$AA?$AA@ 00014448     common.obj
 0002:000002bc       ??_C@_1BI@KGAJ@?$AAR?$AAi?$AAg?$AAh?$AAt?$AAT?$AAr?$AAe?$AAb?$AAl?$AAe?$AA?$AA@ 0001445c     common.obj
 0002:000002d4       ??_C@_1BG@BGGD@?$AAL?$AAe?$AAf?$AAt?$AAT?$AAr?$AAe?$AAb?$AAl?$AAe?$AA?$AA@ 00014474     common.obj
 0002:000002ec       ??_C@_1O@IECC@?$AAM?$AAi?$AAc?$AAA?$AAG?$AAC?$AA?$AA@ 0001448c     common.obj
 0002:000002fc       ??_C@_1CA@EJHI@?$AAR?$AAi?$AAg?$AAh?$AAt?$AAO?$AAu?$AAt?$AAp?$AAu?$AAt?$AAG?$AAa?$AAi?$AAn?$AA?$AA@ 0001449c     common.obj
 0002:0000031c       ??_C@_1BO@PPLI@?$AAL?$AAe?$AAf?$AAt?$AAO?$AAu?$AAt?$AAp?$AAu?$AAt?$AAG?$AAa?$AAi?$AAn?$AA?$AA@ 000144bc     common.obj
 0002:0000033c       ??_C@_1BO@PMCJ@?$AAR?$AAi?$AAg?$AAh?$AAt?$AAI?$AAn?$AAp?$AAu?$AAt?$AAG?$AAa?$AAi?$AAn?$AA?$AA@ 000144dc     common.obj
 0002:0000035c       ??_C@_1BM@CFEM@?$AAL?$AAe?$AAf?$AAt?$AAI?$AAn?$AAp?$AAu?$AAt?$AAG?$AAa?$AAi?$AAn?$AA?$AA@ 000144fc     common.obj
 0002:00000378       ??_C@_1CA@CIKM@?$AAR?$AAi?$AAg?$AAh?$AAt?$AAI?$AAn?$AAp?$AAu?$AAt?$AAM?$AAi?$AAx?$AAe?$AAr?$AA?$AA@ 00014518     common.obj
 0002:00000398       ??_C@_1BO@JOGM@?$AAL?$AAe?$AAf?$AAt?$AAI?$AAn?$AAp?$AAu?$AAt?$AAM?$AAi?$AAx?$AAe?$AAr?$AA?$AA@ 00014538     common.obj
 0002:000003b8       ??_C@_1BI@BMOJ@?$AAO?$AAu?$AAt?$AAp?$AAu?$AAt?$AAM?$AAi?$AAx?$AAe?$AAr?$AA?$AA@ 00014558     common.obj
 0002:000003d0       ??_C@_1BE@GLOL@?$AAP?$AAc?$AAS?$AAp?$AAk?$AAr?$AAV?$AAo?$AAl?$AA?$AA@ 00014570     common.obj
 0002:000003e4       ??_C@_1O@MNBB@?$AAM?$AAi?$AAc?$AAV?$AAo?$AAl?$AA?$AA@ 00014584     common.obj
 0002:000003f4       ??_C@_1BO@HCKE@?$AAR?$AAi?$AAg?$AAh?$AAt?$AAL?$AAi?$AAn?$AAe?$AAI?$AAn?$AAV?$AAo?$AAl?$AA?$AA@ 00014594     common.obj
 0002:00000414       ??_C@_1BM@KLMB@?$AAL?$AAe?$AAf?$AAt?$AAL?$AAi?$AAn?$AAe?$AAI?$AAn?$AAV?$AAo?$AAl?$AA?$AA@ 000145b4     common.obj
 0002:00000430       ??_C@_1BG@COJL@?$AAR?$AAi?$AAg?$AAh?$AAt?$AAC?$AAD?$AAV?$AAo?$AAl?$AA?$AA@ 000145d0     common.obj
 0002:00000448       ??_C@_1BE@KMKA@?$AAL?$AAe?$AAf?$AAt?$AAC?$AAD?$AAV?$AAo?$AAl?$AA?$AA@ 000145e8     common.obj
 0002:0000045c       ??_C@_1BK@JCIM@?$AAR?$AAi?$AAg?$AAh?$AAt?$AAM?$AAi?$AAd?$AAi?$AAV?$AAo?$AAl?$AA?$AA@ 000145fc     common.obj
 0002:00000478       ??_C@_1BI@KBIJ@?$AAL?$AAe?$AAf?$AAt?$AAM?$AAi?$AAd?$AAi?$AAV?$AAo?$AAl?$AA?$AA@ 00014618     common.obj
 0002:00000490       ??_C@_1BK@MFCG@?$AAR?$AAi?$AAg?$AAh?$AAt?$AAW?$AAa?$AAv?$AAe?$AAV?$AAo?$AAl?$AA?$AA@ 00014630     common.obj
 0002:000004ac       ??_C@_1BI@PGCD@?$AAL?$AAe?$AAf?$AAt?$AAW?$AAa?$AAv?$AAe?$AAV?$AAo?$AAl?$AA?$AA@ 0001464c     common.obj
 0002:000004c4       ??_C@_1BO@NHA@?$AAR?$AAi?$AAg?$AAh?$AAt?$AAM?$AAa?$AAs?$AAt?$AAe?$AAr?$AAV?$AAo?$AAl?$AA?$AA@ 00014664     common.obj
 0002:000004e4       ??_C@_1BM@NEBF@?$AAL?$AAe?$AAf?$AAt?$AAM?$AAa?$AAs?$AAt?$AAe?$AAr?$AAV?$AAo?$AAl?$AA?$AA@ 00014684     common.obj
 0002:00000500       ??_7CAdapterCommon@@6BCUnknown@@@ 000146a0     common.obj
 0002:00000510       ??_7CAdapterCommon@@6BIAdapterPowerManagement@@@ 000146b0     common.obj
 0002:00000528       ??_7CAdapterCommon@@6BIAdapterCommon@@@ 000146c8     common.obj
 0002:00000650       ??_7CMiniportTopologyHDA@@6BCUnknown@@@ 000147f0     mintopo.obj
 0002:00000660       ??_7CMiniportTopologyHDA@@6BIMiniportTopology@@@ 00014800     mintopo.obj
 0002:00000678       ??_7CMiniportWaveCyclicHDA@@6BCUnknown@@@ 00014818     minwave.obj
 0002:00000688       ??_7CMiniportWaveCyclicHDA@@6BIMiniportWaveCyclic@@@ 00014828     minwave.obj
 0002:000006a4       ??_7CMiniportWaveCyclicStreamHDA@@6BCUnknown@@@ 00014844     minwave.obj
 0002:000006b4       ??_7CMiniportWaveCyclicStreamHDA@@6BIMiniportWaveCyclicStream@@@ 00014854     minwave.obj
 0002:000006d8       ??_7CUnknown@@6B@          00014878     stdunk:stdunk.obj
 0003:00000000       ?ulDebugOut@@3KA           000148a0     adapter.obj
 0003:00000008       __GUID_b7902fe9_fb0a_11d1_81b0_0060083316c1 000148a8     adapter.obj
 0003:00000018       __GUID_d3f0ce1c_fffc_11d1_81b0_0060083316c1 000148b8     adapter.obj
 0003:00000028       __GUID_c096df9c_fb09_11d1_81b0_0060083316c1 000148c8     adapter.obj
 0003:00000140       ?audBufSize@@3KA           000149e0     common.obj
 0003:00000144       ?BdlSize@@3KA              000149e4     common.obj
 0003:00000840       __GUID_185fedf6_9905_11d1_95a9_00c04fb925d3 000150e0     mintopo.obj
 0003:00000850       __GUID_185fedef_9905_11d1_95a9_00c04fb925d3 000150f0     mintopo.obj
 0003:00000860       __GUID_185fede1_9905_11d1_95a9_00c04fb925d3 00015100     mintopo.obj
 0003:00000870       __GUID_185fede0_9905_11d1_95a9_00c04fb925d3 00015110     mintopo.obj
 0003:00000880       __GUID_7607e580_c557_11d0_8a2b_00a0c9255ac1 00015120     mintopo.obj
 0003:00000890       __GUID_185fede3_9905_11d1_95a9_00c04fb925d3 00015130     mintopo.obj
 0003:000008a0       __GUID_da441a60_c556_11d0_8a2b_00a0c9255ac1 00015140     mintopo.obj
 0003:000008b0       __GUID_185fedee_9905_11d1_95a9_00c04fb925d3 00015150     mintopo.obj
 0003:000008c0       __GUID_02b223c0_c557_11d0_8a2b_00a0c9255ac1 00015160     mintopo.obj
 0003:000008d0       __GUID_185feded_9905_11d1_95a9_00c04fb925d3 00015170     mintopo.obj
 0003:000008e0       __GUID_e88c9ba0_c557_11d0_8a2b_00a0c9255ac1 00015180     mintopo.obj
 0003:000008f0       __GUID_185fedec_9905_11d1_95a9_00c04fb925d3 00015190     mintopo.obj
 0003:00000900       __GUID_185fedeb_9905_11d1_95a9_00c04fb925d3 000151a0     mintopo.obj
 0003:00000910       __GUID_185fedea_9905_11d1_95a9_00c04fb925d3 000151b0     mintopo.obj
 0003:00000920       __GUID_185fede9_9905_11d1_95a9_00c04fb925d3 000151c0     mintopo.obj
 0003:00000930       __GUID_185fede8_9905_11d1_95a9_00c04fb925d3 000151d0     mintopo.obj
 0003:00000940       __GUID_e573adc0_c555_11d0_8a2b_00a0c9255ac1 000151e0     mintopo.obj
 0003:00000950       __GUID_185fede7_9905_11d1_95a9_00c04fb925d3 000151f0     mintopo.obj
 0003:00000960       __GUID_185fede5_9905_11d1_95a9_00c04fb925d3 00015200     mintopo.obj
 0003:00000970       __GUID_3a5acc00_c557_11d0_8a2b_00a0c9255ac1 00015210     mintopo.obj
 0003:00000980       __GUID_45ffaaa0_6e1b_11d0_bcf2_444553540000 00015220     mintopo.obj
 0003:00000990       __GUID_6994ad04_93ef_11d0_a3cc_00a0c9223196 00015230     mintopo.obj
 0003:000009a0       __GUID_185fedf7_9905_11d1_95a9_00c04fb925d3 00015240     mintopo.obj
 0003:000009b0       __GUID_dff21ce1_f70f_11d0_b917_00a0c9223196 00015250     mintopo.obj
 0003:000009c0       __GUID_dff21be1_f70f_11d0_b917_00a0c9223196 00015260     mintopo.obj
 0003:000009d0       __GUID_185fedf9_9905_11d1_95a9_00c04fb925d3 00015270     mintopo.obj
 0003:000009e0       __GUID_dff21fe3_f70f_11d0_b917_00a0c9223196 00015280     mintopo.obj
 0003:000009f0       __GUID_185fedfb_9905_11d1_95a9_00c04fb925d3 00015290     mintopo.obj
 0003:00000a00       __GUID_dff220e3_f70f_11d0_b917_00a0c9223196 000152a0     mintopo.obj
 0003:00000a10       __GUID_185fedf8_9905_11d1_95a9_00c04fb925d3 000152b0     mintopo.obj
 0003:00000a20       __GUID_dff220f3_f70f_11d0_b917_00a0c9223196 000152c0     mintopo.obj
 0003:00000a30       __GUID_dff21fe4_f70f_11d0_b917_00a0c9223196 000152d0     mintopo.obj
 0003:00000a40       __GUID_97e99ba0_bdea_11cf_a5d6_28db04c10000 000152e0     mintopo.obj
 0003:00000c88       __GUID_507ae360_c554_11d0_8a2b_00a0c9255ac1 00015528     minwave.obj
 0003:00000c98       __GUID_4d837fe0_c555_11d0_8a2b_00a0c9255ac1 00015538     minwave.obj
 0003:00000ca8       __GUID_185fedfa_9905_11d1_95a9_00c04fb925d3 00015548     minwave.obj
 0003:00000cb8       __GUID_fb6c4281_0353_11d1_905f_0000c0cc16ba 00015558     minwave.obj
 0003:00000cc8       __GUID_05589f81_c356_11ce_bf01_00aa0055595a 00015568     minwave.obj
 0003:00000cd8       __GUID_00000001_0000_0010_8000_00aa00389b71 00015578     minwave.obj
 0003:00000ce8       __GUID_73647561_0000_0010_8000_00aa00389b71 00015588     minwave.obj
 0003:00000cf8       __GUID_518590a2_a184_11d0_8522_00c04fd9baf3 00015598     minwave.obj
 0003:00000d08       __GUID_0f6417d6_c318_11d0_a43f_00a0c9223196 000155a8     minwave.obj
 0003:00000d18       __GUID_00000000_0000_0000_0000_000000000000 000155b8     adapter.obj
 0004:0000003e       _AddDevice@8               0001561e f   adapter.obj
 0004:0000026a       ?InstallSubdevice@@YGJPAU_DEVICE_OBJECT@@PAU_IRP@@PAGABU_GUID@@3P6GJPAPAUIUnknown@@3PAU4@W4_POOL_TYPE@@@Z5PAUIResourceList@@344@Z 0001584a f   adapter.obj
 0004:0000066e       ?StartDevice@@YGJPAU_DEVICE_OBJECT@@PAU_IRP@@PAUIResourceList@@@Z 00015c4e f   adapter.obj
 0004:00000e6e       ?AssignResources@@YGJPAUIResourceList@@PAPAU1@11111@Z 0001644e f   adapter.obj
 0004:000013c8       ?NewAdapterCommon@@YGJPAPAUIUnknown@@ABU_GUID@@PAU1@W4_POOL_TYPE@@@Z 000169a8 f   common.obj
 0004:00001d49       ?Init@CAdapterCommon@@UAGJPAUIResourceList@@PAU_DEVICE_OBJECT@@@Z 00017329 f   common.obj
 0004:00003252       ??1CAdapterCommon@@UAE@XZ  00018832 f   common.obj
 0004:000036b7       ?NonDelegatingQueryInterface@CAdapterCommon@@UAGJABU_GUID@@PAPAX@Z 00018c97 f   common.obj
 0004:0000380e       ?WavePortDriverDest@CAdapterCommon@@UAGPAPAUIUnknown@@XZ 00018dee f   common.obj
 0004:000038ae       ?GetInterruptSync@CAdapterCommon@@UAGPAUIInterruptSync@@XZ 00018e8e f   common.obj
 0004:0000394e       ?MidiPortDriverDest@CAdapterCommon@@UAGPAPAUIUnknown@@XZ 00018f2e f   common.obj
 0004:000039ee       ?SetWaveServiceGroup@CAdapterCommon@@UAGXPAUIServiceGroup@@@Z 00018fce f   common.obj
 0004:00004102       ?InitHDAController@CAdapterCommon@@QAGJXZ 000196e2 f   common.obj
 0004:00005126       ?InitializeCodec@CAdapterCommon@@QAGJE@Z 0001a706 f   common.obj
 0004:0000582b       ?hda_initialize_audio_function_group@CAdapterCommon@@QAGJKK@Z 0001ae0b f   common.obj
 0004:0000670e       ?hda_get_node_type@CAdapterCommon@@QAGEKK@Z 0001bcee f   common.obj
 0004:000067be       ?hda_get_node_connection_entries@CAdapterCommon@@QAGKKKK@Z 0001bd9e f   common.obj
 0004:000068d0       ?hda_enable_pin_output@CAdapterCommon@@QAGXKK@Z 0001beb0 f   common.obj
 0004:00006910       ?hda_disable_pin_output@CAdapterCommon@@QAGXKK@Z 0001bef0 f   common.obj
 0004:00006950       ?hda_is_headphone_connected@CAdapterCommon@@QAGEXZ 0001bf30 f   common.obj
 0004:00006a52       ?hda_initialize_output_pin@CAdapterCommon@@QAGXK@Z 0001c032 f   common.obj
 0004:00006e76       ?hda_initialize_audio_output@CAdapterCommon@@QAGXK@Z 0001c456 f   common.obj
 0004:0000729a       ?hda_initialize_audio_mixer@CAdapterCommon@@QAGXK@Z 0001c87a f   common.obj
 0004:000075d2       ?hda_initialize_audio_selector@CAdapterCommon@@QAGXK@Z 0001cbb2 f   common.obj
 0004:000078d2       ?ReadRegistryBoolean@CAdapterCommon@@AAGEPBGE@Z 0001ceb2 f   common.obj
 0004:00007ab8       ?CreateMiniportTopologyHDA@@YGJPAPAUIUnknown@@ABU_GUID@@PAU1@W4_POOL_TYPE@@@Z 0001d098 f   mintopo.obj
 0004:00007c2a       ?ProcessResources@CMiniportTopologyHDA@@AAEJPAUIResourceList@@@Z 0001d20a f   mintopo.obj
 0004:00007dba       ?NonDelegatingQueryInterface@CMiniportTopologyHDA@@UAGJABU_GUID@@PAPAX@Z 0001d39a f   mintopo.obj
 0004:00007f6e       ??1CMiniportTopologyHDA@@UAE@XZ 0001d54e f   mintopo.obj
 0004:00008146       ?Init@CMiniportTopologyHDA@@UAGJPAUIUnknown@@PAUIResourceList@@PAUIPortTopology@@@Z 0001d726 f   mintopo.obj
 0004:0000835a       ?GetDescription@CMiniportTopologyHDA@@UAGJPAPAUPCFILTER_DESCRIPTOR@@@Z 0001d93a f   mintopo.obj
 0004:00009b38       ?CreateMiniportWaveCyclicHDA@@YGJPAPAUIUnknown@@ABU_GUID@@PAU1@W4_POOL_TYPE@@@Z 0001f118 f   minwave.obj
 0004:00009e06       ?ProcessResources@CMiniportWaveCyclicHDA@@AAEJPAUIResourceList@@@Z 0001f3e6 f   minwave.obj
 0004:0000a272       ?ValidateFormat@CMiniportWaveCyclicHDA@@AAEJPATKSDATAFORMAT@@@Z 0001f852 f   minwave.obj
 0004:0000a4ae       ?NonDelegatingQueryInterface@CMiniportWaveCyclicHDA@@UAGJABU_GUID@@PAPAX@Z 0001fa8e f   minwave.obj
 0004:0000a662       ??1CMiniportWaveCyclicHDA@@UAE@XZ 0001fc42 f   minwave.obj
 0004:0000a866       ?Init@CMiniportWaveCyclicHDA@@UAGJPAUIUnknown@@PAUIResourceList@@PAUIPortWaveCyclic@@@Z 0001fe46 f   minwave.obj
 0004:0000aafe       ?GetDescription@CMiniportWaveCyclicHDA@@UAGJPAPAUPCFILTER_DESCRIPTOR@@@Z 000200de f   minwave.obj
 0004:0000acea       ?DataRangeIntersection@CMiniportWaveCyclicHDA@@UAGJKPATKSDATAFORMAT@@0KPAXPAK@Z 000202ca f   minwave.obj
 0004:0000b2ea       ?NewStream@CMiniportWaveCyclicHDA@@UAGJPAPAUIMiniportWaveCyclicStream@@PAUIUnknown@@W4_POOL_TYPE@@KEPATKSDATAFORMAT@@PAPAUIDmaChannel@@PAPAUIServiceGroup@@@Z 000208ca f   minwave.obj
 0004:0000b682       ?NonDelegatingQueryInterface@CMiniportWaveCyclicStreamHDA@@UAGJABU_GUID@@PAPAX@Z 00020c62 f   minwave.obj
 0004:0000b82e       ??1CMiniportWaveCyclicStreamHDA@@UAE@XZ 00020e0e f   minwave.obj
 0004:0000baa0       ?Init@CMiniportWaveCyclicStreamHDA@@QAEJPAVCMiniportWaveCyclicHDA@@KEPATKSDATAFORMAT@@PAUIDmaChannel@@@Z 00021080 f   minwave.obj
 0004:0000bd12       ?SetNotificationFreq@CMiniportWaveCyclicStreamHDA@@UAGKKPAK@Z 000212f2 f   minwave.obj
 0004:0000bea6       ?SetFormat@CMiniportWaveCyclicStreamHDA@@UAGJPATKSDATAFORMAT@@@Z 00021486 f   minwave.obj
 0004:0000c0ee       ?SetState@CMiniportWaveCyclicStreamHDA@@UAGJW4KSSTATE@@@Z 000216ce f   minwave.obj
 0005:0000003e       _DriverEntry@8             0002181e f   adapter.obj
 0005:000000ac       __IMPORT_DESCRIPTOR_ntoskrnl 0002188c     ntoskrnl:ntoskrnl.exe
 0005:000000c0       __IMPORT_DESCRIPTOR_HAL    000218a0     hal:HAL.dll
 0005:000000d4       __IMPORT_DESCRIPTOR_portcls 000218b4     portcls:portcls.sys
 0005:000000e8       __NULL_IMPORT_DESCRIPTOR   000218c8     ntoskrnl:ntoskrnl.exe

 entry point at        0005:0000003e

 Static symbols

 0004:000084ae       ?PropertyHandler_OnOff@@YGJPAU_PCPROPERTY_REQUEST@@@Z 0001da8e f   mintopo.obj
 0004:000088c6       ?PropertyHandler_SuperMixCaps@@YGJPAU_PCPROPERTY_REQUEST@@@Z 0001dea6 f   mintopo.obj
 0004:00008ed6       ?PropertyHandler_SuperMixTable@@YGJPAU_PCPROPERTY_REQUEST@@@Z 0001e4b6 f   mintopo.obj
 0004:00009606       ?PropertyHandler_CpuResources@@YGJPAU_PCPROPERTY_REQUEST@@@Z 0001ebe6 f   mintopo.obj
 0001:0000326e       ?PropertyHandler_Level@@YGJPAU_PCPROPERTY_REQUEST@@@Z 0001354e f   mintopo.obj
 0004:00009866       ?BasicSupportHandler@@YGJPAU_PCPROPERTY_REQUEST@@@Z 0001ee46 f   mintopo.obj

 318 bytes saved through ICF

